:020000040000FA
:020000001028C6
:08000800A0000308A10021087B
:080010008300A00E200E090080
:1000200083168F3081009F01960199018B01831205
:100030009F01073099000A30F8224314B30185016B
:100040008316C830850083123430B9001530C200E1
:100050004314051505160230FE22051105128519F7
:100060001B28B30186210A30F82239220330F822F6
:100070002A220330F82239220330F82248221E08AF
:10008000B8000C230A30F8220122FD210A30F822A0
:100090006622B8000C230A30F822FD2101220A3022
:1000A000F822831605110512831205150516023074
:1000B000FE22051105120F30F822851951286421FE
:1000C000C001BD01BE0143120130C200C20B86282F
:1000D0001530C2000508A20005100430FE22482297
:1000E00022080339850487301E02031C862801304C
:1000F000C20040182522401C3922C00A1E210130AE
:10010000F8221E2163006300630066286400431E1A
:100110008C2840181522401C1E22BE0AC00AC52287
:100120006430FE221E304006031943162D3040066F
:10013000031943123C3040060319B5288519662877
:10014000BD0A15220730BD0503303D060319D12035
:1001500004303D060319FA2006303D060319AA2192
:1001600021221430F8221522662805100530831646
:10017000051183120515B9004D210230F8228621A0
:10018000EE2264006300851DC728B90BC2288316C0
:100190000511831205150230F822B30164210511FF
:1001A00060287830AA000F30AB00AC00B8210130D5
:1001B000F822B430AA000F30AB001830AC00CC21CC
:1001C0004630AB002D0805220800B430AA000F30DD
:1001D000AB001830AC00CC210130F8226430AA000A
:1001E0001930AB001430AC00B8215030AB002D08F2
:1001F00005220800EC2106210730FE2206210730E7
:10020000FE2206210730FE220621E1293C30B400FF
:100210004130AB002B08AD00303085060B30A40018
:100220000000000000006400A40B1029AD0B0C2995
:1002300006300423AB03B40B0A2908000C30B300CA
:100240009630AA000A30AB001430AC00B8210A3056
:100250000A30AB001E30AC00CC212D08B30B212995
:100260006430AB002D0805220130F8220800083068
:10027000B1002830AA000F30AB001430AC00B82118
:100280001430B10B39291030B1004630AA000C30BF
:10029000AB00B821B10B452908000830B10032305D
:1002A000AA000F30AB001430AC00CC211430B10BDD
:1002B0004F291030B1005030AA000C30AB00CC21D7
:1002C0001430B10B5B2908002830B1002830AA0097
:1002D0001E30AB001E30AC00CC21AA03B10B682944
:1002E0000800B30A1E30B2001E30AA000F30AB0067
:1002F0000F30AC000230B100CC216400B10B7C297E
:10030000AA03B20B7A29B30B72290800B30A1E3074
:10031000B2000A30AA000C30AB000F30AC00023043
:10032000B100CC216400B10B9129AA0AAA0AB20B30
:100330008F29B30B872908000730B1003230AA009B
:100340003730AB000530AC00B8216430FE22B10B71
:100350009E2908001430B1001930AA000F30AB00FC
:100360000A30AC00B8210A30FE22B10BAC290800DB
:10037000EC212A08AD002B08AE002C08AF002D0898
:10038000A400A40BC12930308506AF0BBF2964003F
:10039000AD03AE0BBD29E129EC212A08AD002B08E5
:1003A000AE002C08AF002D08A400A40BD5293030D6
:1003B0008506AF0BD3296400AD0FDF29AD03AE0B6B
:1003C000D12905128512143004233A0883168500BA
:1003D00085128312851208008316050805128512FE
:1003E0008312BA000516851208003230AB00ED30DA
:1003F000052A6530AB007530052ABE30AB001D30D4
:10040000052AE230AB001830052A6400AA00EC216E
:100410000830B0002A08A400A40B0C2A303085064E
:10042000B00B0A2AAB0B082AE129831605108510A8
:10043000831205100430FE228510080015220514D1
:100440000800152285140514080021220530F82221
:100450001522080021220F30F8221522080021223F
:100460001C30F8221522080021223230F8221522F1
:1004700008001E220530F822152208001E220F3027
:10048000F822152208001E221930F8221522080031
:100490001F14831685109F018312851464009E012A
:1004A0000230FE228316851452309F00831285107D
:1004B00005309F00143004239F140A3004239F1832
:1004C0005D2A83169F0183129F0108001F14831663
:1004D0009F019E010511831205112830FE2283160B
:1004E000051554309F0083126430FE2289309F002E
:1004F000143004239F140A3004239F187B2A831688
:100500009F011E0883129F01080083169F019E0110
:100510008510051105128512831285140511051227
:1005200085122830FE2283168514051505168516BA
:100530005C309F0083126430FE22831685145E3087
:100540009F0083120518C314051CC31005108530C5
:100550009F00143004239F140A3004239F18AC2AF0
:10056000C318051483169F011E0883129F010800FB
:100570008522B80015220530F8220C230530F82218
:100580000122FD210530F82208006622BB003B084D
:1005900004303B02031CD42A431808004314B3015F
:1005A0007121431905140800431CDE2A0518431560
:1005B000051C431105104310B3018621831605085D
:1005C000A30083120508A200EE22630063008316D5
:1005D00023088500831222088500C52A0730990068
:1005E000850183169F01FF30850083128501080075
:1005F000A6002830FE22A60BF92A0800A500FA3032
:100600000423A50BFF2A0800A400062B072B640077
:10061000A403240F052B0800B601B701643038028B
:10062000031C152BB800B60A0E2B0A303802031C27
:100630001C2BB800B70A152B2A230730F8223708DD
:10064000B6002A230730F8223808B6002A230730DC
:10065000F8220800B608031D2F2BF52100340130C5
:0E066000B602031C0034F9210230F8222F2BC1
:1007E0006314B2143018201CF0206C38E534203229
:1007F000EE24F039F234F430EF3473374C164326DC
:02400E008C3FE5
:00000001FF
